:020000040000FA
:06000000FE300D303A282D
:08000800A000030EA100831209
:100010008B10851E4317851AC317210E8300A00E6F
:04002000200E0900A5
:0C007400203084008001840A80300402E7
:10008000031C3C280130E500E300D300E4007E308F
:10009000DC000030F300F400F500F600F700F80093
:1000A0000A30AC004C1083162E30850520308605B2
:1000B0000030870583128501860187011030831681
:1000C0008E008312703083168F0083120030031766
:1000D00099000313003003179A00031300309700B0
:1000E00000309F00003083169F00831200300317FA
:1000F0009E000313003003179F000313C0308316C4
:10010000810083123130900000309200003083165D
:100110009400831200309400A63083169800831256
:10012000003083169B008312903098003330831682
:1001300099008312003083168C00831200308316DE
:100140008D00831250308B008B13063003178D0007
:1001500083168C130C1483120C080313F200F203A1
:1001600081018E018F010B118B100B108C128C01F1
:100170008D018B17D220A723CA2364215818D420BD
:10018000581C10218E228F080319BA288F01F621DE
:10019000CD22AD22AA0BBA28AB0A2B1958142B1961
:1001A0005812BA2864000800D8182D29700AD10006
:1001B000D20139215208D0003E24D40059185417D6
:1001C0005108D0003E24D500D9185517C21FFF286A
:1001D000581EFF280310720C70077202031CF928C6
:1001E0000319F9280310720C023E7007D100D201E6
:1001F00002290310720C7002D100D2010229710A87
:10020000D100D20139215208D0003E24D60059191C
:1002100056175108D0003E24D700D91957170800A7
:10022000720AD100D20139215208D0003E24D400F4
:100230005108D0003E24D5001230D100D20139211E
:100240005208D0003E24D6005108D0003E24D700EA
:1002500054175517561757170800A730D4004908E8
:10026000D0003E24D500D601D7015613D91957170F
:1002700008000A305102031C0800D100D20A3929B3
:10028000531C49294213C2138518C21785194217F6
:100290000800D31C52294211C21185184215851934
:1002A000C2150800531D5B29C21043108518C214E3
:1002B000851943140800D31D08004212C212851884
:1002C00042168519C21608005910D910C4185914BD
:1002D000C41CD914461C6E2940147929401C782965
:1002E0004413441345176614671765236716E7160A
:1002F0004010441B5A15441F5911441F5A114C1CDD
:1003000086295819D915581DD9119029DA157E302A
:10031000DC000030F300F400F500F600F700F80010
:10032000441B5A15441F5911441F5A11431CC31032
:10033000431C9E29C3189E29C3143022C21CC1101D
:10034000C21CAF29C118AF29C1142030C7064810FC
:10035000C8104811C811C816E61467176523421D56
:100360004111421DBE294119BE2941150130C40663
:100370004513C5104514661467176523C21DC111C6
:10038000C21DCF29C119CF29C1150830C706481091
:10039000C8104811C815C812E61467176523421E15
:1003A0004112421EE029411AE02941160130C706D8
:1003B0004814C8104811C811C812E61467176523FD
:1003C000C21EC112C21EF129C11AF129C116023082
:1003D000C7064810C8144811C811C812E614671798
:1003E0006523AD0B08005A08D9060800D81D08007F
:1003F000D8114A08CD054B08CE054E084B06FE0025
:100400004D084A06FF0000307E1B0830FE1A0730F8
:100410007E1A0630FE1905307E190430FE180330AE
:100420007E1802307F180130C90058114A0801397E
:10043000031D58154B087F39031D5815581D2B2ACD
:10044000DB080319262ADB0358110800C908D81055
:10045000031DD8140800C9010530DB00D8100800BE
:10046000D8186A2A441B392A7008710203194E2AC7
:10047000432A44134517C5104510661467176523B2
:100480006716E716080044174517C514451066148B
:100490006615671765236716E71608000310720CC8
:1004A00070077202031C5C2A03195C2A0310720C89
:1004B000013E7007F000612A0310720C013E7002C9
:1004C000F00044134517C5144510661466156717E8
:1004D000652308004908083C03194E174908073CE2
:1004E0000319CE164908063C03194E164908053C67
:1004F0000319CE154908043C03194E154908033C5D
:100500000319CE144908023C03194E144908013C52
:1005100003194D144908083C03194E174021D30D07
:10052000531A531406170616051605148701531C93
:100530009C2A06135408AB2AD31CA12A061255087C
:10054000AB2A531DA62A05125608AB2AD31D080054
:1005500005105708AB2A87000800671F0800E3034F
:10056000031D080065186008E51861086519620830
:1005700099000330E3000310E50DE519C02A0800D7
:100580000F30E3000130E500E6080319C92A6523AE
:10059000080067130130E5000800EB080319D72AAB
:1005A000AC0BD62AEB030A30AC00D82AD82A4C1060
:1005B0008C1E08004C148C30EB000A30AC0018196B
:1005C000CA146908E8006A08E9001A08EA0068081D
:1005D000583C031DF62A6908593C031DF62A6A088F
:1005E0005A3C031DF62A0330EE000800EE0B08000B
:1005F0000330EE006808463C031D062B6908671EA1
:10060000C4006A08671EC6006712602B6808453C74
:10061000031D102B6908CA006A08CB00D815602B8F
:1006200068084C3C031D1B2B6908E71EF000E7120D
:100630006A08F100602B6808413C031D212B15243A
:10064000602B6808473C031D602B15246908103C8B
:1006500003193F2B6908113C0319422B6908123C0E
:100660000319452B6908133C0319482B6908023C00
:1006700003194B2B6908033C03194E2B08006A0829
:10068000F300512B6A08F400512B6A08F500512B36
:100690006A08F600512B6A08F700512B6A08F80027
:1006A000512BC21F08007608F3047708F404780879
:1006B000F5047308F6047408F7047508F8040800D4
:1006C00008000310E40D0318641464086605031998
:1006D000612BE001E101E201E41D742BE611F03031
:1006E000E0006F08E100E201641D7D2B6611C4305B
:1006F000E0007008E1007108E200E41C862BE610BF
:10070000C230E0004708E1004808E200641C8F2B7B
:100710006610C130E0004408E1004508E20008002E
:10072000831203173B088D003A088C0083160317C9
:100730008C130C158B138B1B9A2B55308D00AA3004
:100740008D008C148B170C11831203130800431FA8
:1007500008004313441B08005816AA01AB01C41C2F
:10076000BA2BC410C510C514661467176523671625
:10077000E7160800F00A720A70020318F000ED2371
:10078000FF390319BA2B45106615671765236716DD
:10079000E7160800C31F0800C313441B08005816BF
:1007A000AA01AB01C418DD2BC414C510C51466140E
:1007B000671765236716E7160800F003720AF01B37
:1007C000F007ED23FF390319DD2B4513451066159E
:1007D000671765236716E7160800FF38421F0800F1
:1007E00070080739FE000130FF000130FE02031CD3
:1007F000FC2B0310FF0DF52B70087839FE00031059
:10080000FE0CFE0CFE0C7308FE0303197408FE03B5
:1008100003197508FE0303197608FE030319770808
:10082000FE03031978087F050800DC080319080097
:10083000E608031D0800DC1C202CDC101030392CCD
:100840005C1D252C5C111130392CDC1D2A2CDC118F
:100850001230392C5C1E2F2C5C121330392CDC1E0C
:10086000342CDC120230392C5C1F392C5C13033021
:0C087000392CEF00E6156717652308001F
:100A00000A3050020318D00105308A0050088207CE
:100A10003F341834B634BC349934AD34AF34383440
:040A2000BF34BD34EE
:084000000A00000001000800A5
:02400E00CC03E1
:10420000000001000200AA00C80014003000FF00F6
:104210000000FF00FF00FF00410058001400FF00F5
:104220000000110012001300140015001600170002
:10423000060019001200FF00FF00FF00FF00FF0052
:10424000FF00FF00FF00FF00FF00FF00FF00FF0076
:10425000FF00FF00FF00FF00FF00FF00FF00FF0066
:10426000FF00FF00FF00FF00FF00FF00FF00FF0056
:10427000FF00FF00FF00FF00FF00FF00FF00FF0046
:10428000FF00FF00FF00FF00FF00FF00FF00FF0036
:10429000FF00FF00FF00FF00FF00FF00FF00FF0026
:1042A000FF00FF00FF00FF00FF00FF00FF00FF0016
:1042B000FF00FF00FF00FF00FF00FF00FF00FF0006
:1042C000FF00FF00FF00FF00FF00FF00FF00FF00F6
:1042D000FF00FF00FF00FF00FF00FF00FF00FF00E6
:1042E000FF00FF00FF00FF00FF00FF00FF00FF00D6
:1042F000FF00FF00FF00FF00FF00FF00FF00FF00C6
:00000001FF
